:020000040000FA
:1000000083EF19F012001200C3EF01F0120001009B
:1000100052330000000F0000370000000F0E93164F
:1000200081160ED9939493968194819609D90F0ED7
:100030008114816E300E8110816E2BD801D90F0E84
:100040008116300E811225D8FBD80F0E8116300E86
:10005000811246D91ED819D90F0E811641D9818A2D
:100060003FD917D8280EE66E19D8E552080EE66E6D
:1000700015D8E552010EE66E11D8E552060EE66E71
:100080000DD8E5520C0EE66E09D8E55229D900D0FC
:100090001200818625D981966AEF01F0D9CFE6FF5B
:1000A000E1CFD9FF1DD9819481960F0E8116FE0EE6
:1000B000DB50F00B811214D9ECDF0F0E8116FE0E0F
:1000C000DB38F00BF00B81120BD9E3DF00D0E552E7
:1000D000E7CFD9FF1200D9CFE6FFE1CFD9FF00D992
:1000E000818481960F0E8116FE0EDB50F00B81127B
:1000F0008186F6D881960F0E8116FE0EDB38F00B46
:10010000F00B81128186ECD8819600D0E552E7CFC2
:10011000D9FF1200D9CFE6FFE1CFD9FFFD0EDBCF2B
:10012000F6FFFE0EDBCFF7FF0800F55011E0FD0EE5
:10013000DBCFF6FFFE0EDBCFF7FF0800F550E66ED3
:10014000CADFE552FD0EDB2AFE0E01E3DB2AE6D70D
:1001500000D0E552E7CFD9FF1200D9CFE6FFE1CFBB
:10016000D9FFFD0EDBCFE9FFFE0EDBCFEAFFEF503C
:1001700010E0FD0EDBCFE9FFFE0EDBCFEAFFEF5014
:10018000E66EA9DFE552FD0EDB2AFE0E01E3DB2A57
:10019000E8D700D0E552E7CFD9FF1200D9CFE6FF6C
:1001A000E1CFD9FFE652FE0EDB0404E1FD0EDB5089
:1001B000800FDF6EFE0EDB50020804E1FD0EDB5007
:1001C000C00FDF6EDFCFE6FF69DFE552E552E55293
:1001D000E7CFD9FF1200D9CFE6FFE1CFD9FF020E5A
:1001E000E126E66AFE0EDBCFE6FFD8DFE552E552F8
:1001F000DE6ADD6ADECF14F0DDCF15F0D890155041
:1002000004E6100E145C000E155809E2200EE66E8E
:1002100062DFE552DF2A010E01E3DB2AEBD7E66A53
:10022000FE0EDBCFE6FFBADFE552E552020EE15CDF
:1002300002E2E16AE552E16EE552E7CFD9FF120032
:10024000D9CFE6FFE1CFD9FF020EE126DE6ADD6AF3
:10025000DECF14F0DDCF15F0D890155004E6100E67
:10026000145C270E155806E20000DF2A010E01E398
:10027000DB2AEED700D0020EE15C02E2E16AE55231
:10028000E16EE552E7CFD9FF1200D9CFE6FFE1CF0B
:10029000D9FF020EE126DE6ADD6ADECF14F0DDCF83
:1002A00015F0D890155004E6C40E145C090E1558CC
:1002B00006E20000DF2A010E01E3DB2AEED700D0C0
:1002C000020EE15C02E2E16AE552E16EE552E7CF3F
:1002D000D9FF120000000000000000000000120022
:1002E000D9CFE6FFE1CFD9FF020EE126DE6ADD6A53
:1002F000DECF14F0DDCF15F0D890155004E6E80EEF
:10030000145C030E155806E20000DF2A010E01E31B
:10031000DB2AEED700D0020EE15C02E2E16AE55290
:10032000E16EE552E7CFD9FF1200D9CFE6FFE1CF6A
:10033000D9FF81940F0E8116FE0EDB504009F00BA1
:100340008112C8DFA6DE0F0E8116FE0EDB38F00B21
:10035000F00B8112BFDF9DDE00D0E552E7CFD9FF61
:10036000120000000000000000000000000000007B
:10037000000000000000000000000000000000007D
:10038000000000001200DACFE4FFE2CFDAFFE6520D
:100390009EA007D001012C2B000E2D232E232F23EE
:1003A0009E90E552E5CFDAFF1100D9CFE6FFE1CF0D
:1003B000D9FF020EE126DE6ADD6AFD0EDBCFE9FF22
:1003C000FE0EDBCFEAFFEF5016E0FD0EDBCFE9FFBC
:1003D000FE0EDBCFEAFFEF50E66EE66A1FD8E5526D
:1003E000E552DF2A010E01E3DB2AFD0EDB2AFE0EB9
:1003F00001E3DB2AE2D7DECF14F0DDCF15F014C025
:10040000F3FF15C0F4FF020EE15C03E200D0E16AE5
:10041000E552E16EE552E7CFD9FF1200D9CFE6FFF2
:10042000E1CFD9FFACA2FED7FD0EDBCFE6FF35EC66
:1004300019F0E552E552E7CFD9FF1200D9CFE6FF18
:10044000E1CFD9FF020EE12601013E0E906F010EB1
:10045000916F90C1E6FF91C1E6FFD950FB0FE96EA5
:10046000FF0EDA20EA6EEECFE6FFEECFE6FFEECF2C
:10047000E6FFEFCFE6FF42EC16F0146E060EE15EEB
:10048000145090C1E6FF91C1E6FF8FDFE552E552BF
:10049000F3CFDEFFF4CFDDFF020EE15C02E2E16AA2
:1004A000E552E16EE552E7CFD9FF1200D9CFE6FF62
:1004B000E1CFD9FFD950FB0FE96EFF0EDA20EA6ECB
:1004C000D880000EEE54000EEE54000EEE54000ED6
:1004D000EE540CE2D950FB0FE96EFF0EDA20EA6E03
:1004E000EE06000EEE5AEE5AEE5AE4D7E552E7CF8A
:1004F000D9FF1200D9CFE6FFE1CFD9FF0E0EE126DA
:10050000F90EDBCFDEFFDBCFDDFFF80EDB5000089E
:1005100002E3070E08D0F80EDB50160802E2170EB1
:1005200002D0F80EDB28E66ED950080FE96EDACF5C
:10053000EAFFE552E750EE6EED6A020EDB6A030E4B
:10054000DB6AFB0EDBCF14F0FC0EDBCF15F0FD0EEB
:10055000DBCF16F0FE0EDBCF17F00A6A0B6A0C6ACF
:100560000D6A14C005F015C006F016C007F017C0DC
:1005700008F0E4EC13F0010A33E1F90EDBCFE9FFF8
:10058000DB2AFA0EDBCFEAFF01E3DB2A2D0EEF6E4A
:10059000FB0EDBCF14F0FC0EDBCF15F0FD0EDBCF36
:1005A00016F0FE0EDBCF17F00A6A0B6A800E0C6E97
:1005B000BF0E0D6E14C005F015C006F016C007F092
:1005C00017C008F03FEC13F0FB0E05C0DBFFFC0E7C
:1005D00006C0DBFFFD0E07C0DBFFFE0E08C0DBFF21
:1005E000FB0EDBCF14F0FC0EDBCF15F0FD0EDBCFE6
:1005F00016F0FE0EDBCF17F00A6A0B6A0C6A0D6A62
:1006000014C005F015C006F016C007F017C008F0BA
:10061000DBEC13F0010A4AE1FB0EDBCF14F0FC0E19
:10062000DBCF15F0FD0EDBCF16F0FE0EDBCF17F0A3
:100630000A6A0B6A800E0C6E3F0E0D6E14C005F038
:1006400015C006F016C007F017C008F0E4EC13F070
:10065000010A2CE1146A156A200E166E410E176EFF
:10066000D950FB0FE96EFF0EDA20EA6EEECF05F0EF
:10067000EECF06F0EECF07F0EFCF08F014C00AF08F
:1006800015C00BF016C00CF017C00DF03FEC13F0C6
:1006900008C0EDFF07C0EDFF06C0EDFF05C0EFFF8E
:1006A000020EDB06030E01E2DB06B6D7FB0EDBCF44
:1006B00014F0FC0EDBCF15F0FD0EDBCF16F0FE0EB6
:1006C000DBCF17F00A6A0B6A200E0C6E410E0D6E1E
:1006D00014C005F015C006F016C007F017C008F0EA
:1006E000E4EC13F0010A2EE0FB0EDBCF14F0FC0E5D
:1006F000DBCF15F0FD0EDBCF16F0FE0EDBCF17F0D3
:100700000A6A0B6A200E0C6E410E0D6E14C005F0C5
:1007100015C006F016C007F017C008F0ECEC12F098
:10072000FB0E05C0DBFFFC0E06C0DBFFFD0E07C0A5
:10073000DBFFFE0E08C0DBFF020EDB2A030E01E327
:10074000DB2AB4D7020EDBCF14F0030EDBCF15F09B
:10075000D950080FE96EDACFEAFF1450EE26155093
:10076000ED22010EF36E040EF3CFDBFF050EDB6A04
:10077000040EDBCF06F0050EDBCF07F027EC12F0FE
:100780000A0E05C0DBFF0B0E06C0DBFF0C0E07C018
:10079000DBFF0D0E08C0DBFF040EDBCF14F0050EEF
:1007A000DBCF15F0080EDBCF16F0090EDBCF17F00C
:1007B00015501718E8AE02D0173404D01650145C48
:1007C000175015582EE20A0EDBCF14F00B0EDBCFBC
:1007D00015F00C0EDBCF16F00D0EDBCF17F00A6A0A
:1007E0000B6A200E0C6E410E0D6E14C005F015C084
:1007F00006F016C007F017C008F0ECEC12F00A0E75
:1008000005C0DBFF0B0E06C0DBFF0C0E07C0DBFFD5
:100810000D0E08C0DBFF040EDB2A050E01E3DB2A08
:10082000BBD70A0EDBCF18F00B0EDBCF19F00C0E86
:10083000DBCF1AF00D0EDBCF1BF00A6A0B6A0C6AD5
:10084000400E0D6E18C005F019C006F01AC007F072
:100850001BC008F0ECEC12F005C014F006C015F057
:1008600007C016F008C017F0D950FB0FE96EFF0E55
:10087000DA20EA6EEECF05F0EECF06F0EECF07F00D
:10088000EFCF08F014C00AF015C00BF016C00CF042
:1008900017C00DF056EC12F008C0EDFF07C0EDFFD9
:1008A00006C0EDFF05C0EFFFFB0EDBCF14F0FC0E22
:1008B000DBCF15F0FD0EDBCF16F0FE0EDBCF17F011
:1008C0000A6A0B6A200E0C6E410E0D6E14C005F004
:1008D00015C006F016C007F017C008F0E4EC13F0DE
:1008E000010A13E0FB0EDB6AFC0EDB6A800EF36E7E
:1008F000FD0EF3CFDBFF3F0EF36EFE0EF3CFDBFFFB
:10090000020EDB2A030E01E3DB2A020EDBCF14F01A
:10091000030EDBCF15F00001800E15145FE0F90E19
:10092000DBCFE9FFDB2AFA0EDBCFEAFF01E3DB2AAC
:10093000300EEF6EF90EDBCFE9FFDB2AFA0EDBCFCC
:10094000EAFF01E3DB2A2E0EEF6E080EDBCF14F078
:10095000090EDBCF15F0800E151414E0020EDBCF6C
:1009600016F0030EDBCF17F0080EDB50165C146E8A
:10097000090EDB501758156E020E14C0DBFF030E74
:1009800015C0DBFF040EDB68050EDB68040EDBCF51
:1009900014F0050EDBCF15F0020EDBCF16F0030EC0
:1009A000DBCF17F017501518E8AE02D0153404D07D
:1009B0001450165C1550175811E2F90EDBCFE9FF01
:1009C000DB2AFA0EDBCFEAFF01E3DB2A300EEF6E03
:1009D000040EDB06050E01E2DB06D8D7040EDB6A47
:1009E000050EDB6A040EDBCF14F0050EDBCF15F02D
:1009F000080EDBCF16F0090EDBCF17F015501718D5
:100A0000E8AE02D0173404D01650145C17501558B5
:100A100001E3ACD0FB0EDBCF05F0FC0EDBCF06F024
:100A2000FD0EDBCF07F0FE0EDBCF08F0ACEC13F0D1
:100A3000060E06C0DBFF070E07C0DBFF300EE76EB9
:100A4000060EDBCF14F0070EDBCF15F0E7501426AF
:100A5000000E1522F90EDBCFE9FFDB2AFA0EDBCF01
:100A6000EAFF01E3DB2A14C0EFFF040EDBCF14F032
:100A7000050EDBCF15F0020EDB50141803E1030E58
:100A8000DB5015180BE1F90EDBCFE9FFDB2AFA0E7C
:100A9000DBCFEAFF01E3DB2A2C0EEF6E060EDBCF85
:100AA00006F0070EDBCF07F027EC12F00A0E05C0A8
:100AB000DBFF0B0E06C0DBFF0C0E07C0DBFF0D0ECD
:100AC00008C0DBFF05C014F006C015F007C016F023
:100AD00008C017F0D950FB0FE96EFF0EDA20EA6E5E
:100AE000EECF05F0EECF06F0EECF07F0EFCF08F037
:100AF00014C00AF015C00BF016C00CF017C00DF0B2
:100B000055EC12F008C0EDFF07C0EDFF06C0EDFF89
:100B100005C0EFFF146A156A200E166E410E176E9F
:100B2000D950FB0FE96EFF0EDA20EA6EEECF05F02A
:100B3000EECF06F0EECF07F0EFCF08F014C00AF0CA
:100B400015C00BF016C00CF017C00DF03FEC13F001
:100B500008C0EDFF07C0EDFF06C0EDFF05C0EFFFC9
:100B6000040EDB2A050E01E3DB2A3CD7F90EDBCFAE
:100B7000E9FFFA0EDBCFEAFFEF6A0E0EE15C02E25C
:100B8000E16AE552E16EE552E7CFD9FF12000D0EA2
:100B9000E66EE66A43DCE552E5520A0EE66EE66A68
:100BA0003DDCE552E55212000F01030E386F070ECF
:100BB000926E92989296806A396B8168936AF19EE0
:100BC00061683A6B9468948094829484949C948E27
:100BD000D09C606A1200800E066E250E076E0650CD
:100BE00002E1C20E071824E0065002E1960E071833
:100BF0001AE0065002E14B0E071810E0800E0618AE
:100C000002E1250E071805E0820E0101006F016B5D
:100C100014D0820E0101006F016B0FD0400E010154
:100C2000006F016B0AD0200E0101006F016B05D02F
:100C30000A0E0101006F016B00D0400E006F016BC6
:100C400000C1E6FF01C1E6FF7C0EE66E2AEC18F05B
:100C5000E552E552E5529D989D9AF29CF29E120053
:100C60000F0149914993BD96BD84BD92BD80BF6A75
:100C7000BE6A9E949D941200D596D584D582D59057
:100C8000D59AD59C6A0EE66E670EE66E19EC19F0E1
:100C9000E552E552F294F29AD59E12009480CD6A04
:100CA000CD82CD9ACD98CD96CD94CD8ECD9CCD9044
:100CB000CC6A1200100EE66E270EE66EE66AE66A51
:100CC00056EC02F0E552E552E552E5526DDF83DF66
:100CD0009EAA05D0BFEC18F00101186FF9D70C0ED1
:100CE000E66EE66A0EEC02F0E552E552900EE66E14
:100CF000D00EE66E030EE66EE66A56EC02F0E552A2
:100D0000E552E552E5520101226B236B050E225D8F
:100D1000000E235938E23E0E8E6F010E8F6F22C1F6
:100D2000E9FF23C1EAFF010ED890E936EA36E8066A
:100D3000FBE1000EE9260F0EEA22EECF14F0EFCF12
:100D400015F0166A14C0E6FF15C0E6FF16C0E6FFF0
:100D50008EC1E6FF8FC1E6FF9CEC17F0176E050E03
:100D6000E15E17508EC1E6FF8FC1E6FFD5EC01F0C2
:100D7000E552E552F3CF26F1F4CF27F10101222B02
:100D8000000E2323C3D70EEC00F0010EE66E4EECEE
:100D900000F0E552880EE66E130EE66EE66AE66A2D
:100DA00056EC02F0E552E552E552E55201013E0EE5
:100DB0008E6F010E8F6F226B236B050E225D000E6E
:100DC00023592DE2800EE66E4EEC00F0E55222C172
:100DD000E9FF23C1EAFF010ED890E936EA36E806BA
:100DE000FBE10E0EE9260F0EEA22EECFE6FFEFCF73
:100DF000E6FF8AEC00F0E552E552F00EE66E490E91
:100E0000E66E020EE66EE66A56EC02F0E552E55238
:100E1000E552E5520101222B000E2323CED72CDF11
:100E20003DDFBD6AF28C9D90F29EF29C80A426D09C
:100E3000010E0101306F316B0ACF14F00BCF15F0AA
:100E4000166A14C0E6FF15C0E6FF16C0E6FF8EC1A5
:100E5000E6FF8FC1E6FF9CEC17F0176E050EE15E12
:100E600017508EC1E6FF8FC1E6FFD5EC01F0E552C9
:100E7000E552F3CF26F1F4CF27F125D0040E01017E
:100E8000306F316B0CCF14F00DCF15F0166A14C013
:100E9000E6FF15C0E6FF16C0E6FF8EC1E6FF8FC174
:100EA000E6FF9CEC17F0176E050EE15E17508EC141
:100EB000E6FF8FC1E6FFD5EC01F0E552E552F3CF36
:100EC00026F1F4CF27F163DE01013A6B3B6B1E6B19
:100ED0001F6B0F01366B01012C6B2D6B2E6B2F6B73
:100EE000326B336B366B376B346B356BCD906A0E70
:100EF000E66E670EE66E19EC19F0E552E552000E4B
:100F0000E66EE66AFDEC18F0E552E5529E9AF29420
:100F1000D08E9E9080A405D0010E0101306F316B00
:100F200004D0040E0101306F316BF29CF28E0F0180
:100F3000226B236BF29AF2949D80D58E8986CD80A8
:100F4000F2A4FED70101226B236B040E225D000E7A
:100F5000235904E2222B000E2323F7D7010E0F01A1
:100F60002225226F000E2321236FF2946A0EE66E73
:100F7000670EE66E19EC19F0E552E55201013051A9
:100F80000F01225D010131510F012359D9E38996E7
:100F9000D59ECD90DEEC18F0F3CF32F1F4CF33F1E3
:100FA000F294F29AF29E32C106F033C107F025ECBA
:100FB00012F005C00BF106C00CF107C00DF108C01E
:100FC0000EF12CC104F02DC105F02EC106F02FC189
:100FD00007F03AEC12F005C014F006C015F007C097
:100FE00016F008C017F00A6A0B6A800E0C6E470EE6
:100FF0000D6E14C005F015C006F016C007F017C03E
:1010000008F03FEC13F005C003F106C004F107C07F
:1010100005F108C006F103C10AF004C10BF005C1D7
:101020000CF006C10DF00BC105F00CC106F00DC1AE
:1010300007F00EC108F056EC12F005C007F106C02B
:1010400008F107C009F108C00AF1800EE66E4EEC07
:1010500000F0E55201013E0E8E6F010E8F6F010E02
:101060003A193A6F0A6A600E0B6EEA0E0C6E460E63
:101070000D6E07C105F008C106F009C107F00AC1ED
:1010800008F0E4EC13F0010A04E1010E01013A6FEB
:101090003B6B01013B3504E23A510008000E3B5521
:1010A00001E382D180B436D00A6A0B6A800E0C6EDE
:1010B000400E0D6E07C105F008C106F009C107F02A
:1010C0000AC108F0ECEC12F005C007F106C008F107
:1010D00007C009F108C00AF1010EE66E8EC1E6FFF5
:1010E0008FC1E6FF07C1E6FF08C1E6FF09C1E6FFC1
:1010F0000AC1E6FF7AEC02F0146E070EE15E1450AE
:10110000340EE66E6BEC00F0E552080E01012A6F1A
:101110002B6B34D0310EE66E6BEC00F0E552010E15
:10112000E66E8EC1E6FF8FC1E6FF07C1E6FF08C18C
:10113000E6FF09C1E6FF0AC1E6FF7AEC02F0146E91
:10114000070EE15E14508EC1E6FF8FC1E6FFB5ECDD
:1011500017F0E552E552F3CF26F1F4CF27F1010164
:10116000020E265F000E275B3E0E2625E96E010E5D
:101170002721EA6EEF6A060E2A6F2B6B530EE66E7E
:101180006BEC00F0E552460EE66EE66A0EEC02F0FD
:10119000E552E552720EE66EE66A0EEC02F0E5529A
:1011A000E552650EE66EE66A0EEC02F0E552E55297
:1011B000710EE66EE66A0EEC02F0E552E5523D0E67
:1011C000E66EE66A0EEC02F0E552E552200EE66E9F
:1011D000E66A0EEC02F0E552E5528EC1E6FF8FC1E1
:1011E000E6FFB5EC17F0E552E552F3CF26F1F4CF68
:1011F00027F10101286B296B246B256B26512A5D91
:1012000027512B5929E226512A5D27512B5919E2E2
:101210003E0E2425E96E010E2521EA6EEF50E66EA2
:10122000240E2825E96E0F0E2921EA6EE552E750BB
:10123000EF6E2607000E275B242B2523282B29235E
:10124000E2D7240E2825E96E0F0E2921EA6E2E0E14
:10125000EF6E282B000E2923030E2A5F000E2B5B56
:1012600026512A5D27512B5929E226512A5D275103
:101270002B5919E23E0E2425E96E010E2521EA6E56
:10128000EF50E66E240E2825E96E0F0E2921EA6E36
:10129000E552E750EF6E2607000E275B242B25232F
:1012A000282B2923E2D7240E2825E96E0F0E2921A9
:1012B000EA6E2E0EEF6E282B000E2923030E2A5FF6
:1012C000000E2B5B26512A5D27512B591FE2000E81
:1012D000D8802655000E275519E23E0E2425E96ECA
:1012E000010E2521EA6EEF50E66E240E2825E96EE8
:1012F0000F0E2921EA6EE552E750EF6E2607000E29
:10130000275B242B2523282B2923E1D7240E2825EE
:10131000E96E0F0E2921EA6E480EEF6E282B000EA3
:101320002923240E2825E96E0F0E2921EA6E7A0E54
:10133000EF6E282B000E2923240E2825E96E0F0EB0
:101340002921EA6EEF6A240EE66E0F0EE66EB5EC0A
:1013500017F0E552E552F3CF26F1F4CF27F1010162
:101360000E0E265D000E27590AE2200EE66E6BEC8B
:1013700000F0E5520101262B000E2723F0D7240EA2
:10138000E66E0F0EE66EADEC00F0E552E552240E6F
:10139000E66E0F0EE66ED5EC01F0E552E552F3CFA6
:1013A00026F1F4CF27F1ECD180B418D00A6A0B6A89
:1013B000800E0C6E400E0D6E07C105F008C106F0E0
:1013C00009C107F00AC108F0ECEC12F005C007F102
:1013D00006C008F107C009F108C00AF1180E146E22
:1013E0000D0E156E8F0E166E4D0E176E07C10AF09C
:1013F00008C10BF009C10CF00AC10DF014C005F0D2
:1014000015C006F016C007F017C008F0ECEC12F09B
:1014100005C00BF106C00CF107C00DF108C00EF1BC
:10142000020EE66E8EC1E6FF8FC1E6FF0BC1E6FF3E
:101430000CC1E6FF0DC1E6FF0EC1E6FF7AEC02F03B
:10144000146E070EE15E14500A6A600E0B6EEA0E0F
:101450000C6E460E0D6E07C105F008C106F009C1FD
:1014600007F00AC108F0E4EC13F0010A47E00A6A49
:10147000E60E0B6EAA0E0C6E480E0D6E07C105F03F
:1014800008C106F009C107F00AC108F0E4EC13F046
:10149000010A34E18EC1E6FF8FC1E6FF090EE66E58
:1014A000E66AB40E146E320E156E166A14C0E6FFAC
:1014B00015C0E6FF16C0E6FFFE0EE66EE6684EECCF
:1014C00017F0176E090EE15E1750F3CF26F1F4CF37
:1014D00027F1470EE66E6BEC00F0E5522E0EE66E3D
:1014E0006BEC00F0E5524F0EE66E6BEC00F0E5524F
:1014F0002E0EE66E6BEC00F0E552A0D00A6A240EC8
:101500000B6EF40E0C6E480E0D6E07C105F008C18F
:1015100006F009C107F00AC108F0E4EC13F0010A73
:1015200047E00A6A1B0E0B6EB70E0C6E490E0D6E6D
:1015300007C105F008C106F009C107F00AC108F0AB
:10154000E4EC13F0010A34E18EC1E6FF8FC1E6FF3F
:10155000090EE66EE66AA60E146E320E156E166A57
:1015600014C0E6FF15C0E6FF16C0E6FFFE0EE66EED
:10157000E6684EEC17F0176E090EE15E1750F3CFD8
:1015800026F1F4CF27F1500EE66E6BEC00F0E55239
:101590002E0EE66E6BEC00F0E5524F0EE66E6BEC35
:1015A00000F0E5522E0EE66E6BEC00F0E55246D0F0
:1015B0000A6A1B0E0B6EB70E0C6E490E0D6E07C13C
:1015C00005F008C106F009C107F00AC108F0DBEC1C
:1015D00013F0010A33E18EC1E6FF8FC1E6FF090E69
:1015E000E66EE66A980E146E320E156E166A14C018
:1015F000E6FF15C0E6FF16C0E6FFFE0EE66EE668E3
:101600004EEC17F0176E090EE15E1750F3CF26F17E
:10161000F4CF27F14F0EE66E6BEC00F0E5522E0E84
:10162000E66E6BEC00F0E552430EE66E6BEC00F0FC
:10163000E5522E0EE66E6BEC00F0E552C7EC05F0BD
:101640008EC1E6FF8FC1E6FFB5EC17F0E552E5521B
:10165000F3CF26F1F4CF27F1060E01012A6F2B6B91
:10166000286B296B246B256B26512A5D27512B593A
:1016700029E226512A5D27512B5919E23E0E2425D5
:10168000E96E010E2521EA6EEF50E66E240E282544
:10169000E96E0F0E2921EA6EE552E750EF6E26073C
:1016A000000E275B242B2523282B2923E2D7240E89
:1016B0002825E96E0F0E2921EA6E2E0EEF6E282BDB
:1016C000000E2923030E2A5F000E2B5B26512A5D94
:1016D00027512B591FE2000ED8802655000E2755A2
:1016E00019E23E0E2425E96E010E2521EA6EEF5027
:1016F000E66E240E2825E96E0F0E2921EA6EE552CA
:10170000E750EF6E2607000E275B242B2523282B9E
:101710002923E1D7240E2825E96E0F0E2921EA6E30
:101720004D0EEF6E282B000E2923240E2825E96E7E
:101730000F0E2921EA6EEF6A240EE66E0F0EE66E9A
:10174000B5EC17F0E552E552F3CF26F1F4CF27F1CF
:1017500001010C0E265D000E27590AE2200EE66EEE
:101760006BEC00F0E5520101262B000E2723F0D789
:10177000240EE66E0F0EE66EADEC00F0E552E5527B
:1017800001011E2B000E1F23090ED8801E55000ECE
:101790001F5547E21E6B1F6B80A422D00ACF14F0A6
:1017A0000BCF15F0166A14C0E6FF15C0E6FF16C091
:1017B000E6FF8EC1E6FF8FC1E6FF9CEC17F0176EC7
:1017C000050EE15E17508EC1E6FF8FC1E6FFD5EC36
:1017D00001F0E552E552F3CF26F1F4CF27F121D005
:1017E0000CCF14F00DCF15F0166A14C0E6FF15C02B
:1017F000E6FF16C0E6FF8EC1E6FF8FC1E6FF9CEC58
:1018000017F0176E050EE15E17508EC1E6FF8FC10F
:10181000E6FFD5EC01F0E552E552F3CF26F1F4CF27
:1018200027F169EF07F0120050EC11F0FB0EDBCF4F
:10183000F3FFDB06F35000090AE09EEC11F0FA0E0C
:1018400009EC12F0F3E1151CF1E1010E01D0000EDC
:101850007FEF11F050EC11F03B0EE12402E3E16860
:10186000E652E16E010EDB6A020EDB6AF90EDBCF97
:10187000F6FFFA0EDBCFF7FFFB0EDBCFF8FF080019
:10188000F550DF6EDF5002E1A3EF10F0250EDF5CB4
:1018900002E096EF10F0030EDB6A040EDB6A050E21
:1018A000DB6A060EDB6A070EDB6AB8EC10F02D0E61
:1018B000DF5C0CE02B0EDF5C09E0200EDF5C06E055
:1018C000230EDF5C03E0300EDF5C1AE1DF50300AEC
:1018D00014E0130A0FE0030A0AE00B0A05E0060A07
:1018E000E4E1030EDB80E1D7030EDB82DED7030EDB
:1018F000DB84DBD7030EDB86D8D7030EDB88D5D796
:101900002A0EDF5C1BE1B4EC10F002EC11F010E0E9
:10191000030EDB8006680768130EDBCF0BF0140E96
:10192000DBCF0CF0C8EC14F0040E04C0DBFF03D0D6
:10193000130EEBEC10F0B8EC10F00BD0090EDB6AD4
:1019400059EC11F003E0CDEC11F0FAD7090EEBECF5
:1019500010F0030EDBB0DB982E0EDF5C1BE1B8EC61
:1019600010F02A0EDF5C0BE1B4EC10F002EC11F089
:1019700003E1130E3DEC11F0B8EC10F00BD0090EA2
:10198000DB6A59EC11F003E0CDEC11F0FAD7090E47
:101990003DEC11F0680EDF5C07E1B8EC10F0680E6A
:1019A000DF5C1DE1030E18D0740EDF5C17E07A0EC9
:1019B000DF5C14E0480EDF5C06E0540EDF5C03E001
:1019C0005A0EDF5C02E1020E07D06C0EDF5C03E012
:1019D0006A0EDF5C04E1010E90EC11F0C9DBDF5010
:1019E0006E0A01E17FD31E0A01E192D1200A01E1D2
:1019F0008FD13F0A01E149D11A0A01E146D10D0A0E
:101A000001E143D1200A01E140D13A0A01E13DD18F
:101A1000200A01E13AD1260A01E135D10D0A01E19E
:101A200032D11A0A01E1D9D0200A4AE0300A1FE077
:101A3000460A0EE0250A01E083D3D950F90FE96E7A
:101A4000FF0EDA20EA6E010EEE5E000EEE5AEE5A3E
:101A50009EEC11F0250EE66E95DB03E1151C01E10D
:101A600069D39AEC11F001E26BD3DB2A69D3080E3B
:101A7000DB6A040EDB50010806E2040EDB0462ECB4
:101A800011F0DB508BDB080EDB5009E0030EDB505E
:101A9000010B05E172DB01E04DD3080EDB6A64DB6C
:101AA000EFCFDFFF12EC12F003E1151C01E142D38E
:101AB0009AEC11F001E3DB2A60DB01E141D33AD378
:101AC000070EDB5002080FE1DEEC11F0030EA5EC6F
:101AD00011F00E0EEECFDBFF0F0EEECFDBFF100E80
:101AE000EECFDBFF20D0F70EDBCF17F0F80EDBCF09
:101AF00018F0020E175E000E185AF70E17C0DBFF23
:101B0000F80E18C0DBFF17C0E9FF18C0EAFF95EC1C
:101B100011F0166A0E0E14C0DBFF0F0E15C0DBFFAE
:101B2000100E16C0DBFF0E0EDBCFE6FF0F0EDBCF75
:101B3000E6FF100EDBCFE6FFC3EC17F0E552E552EF
:101B4000E552130E05C0DBFF140E06C0DBFF060EC8
:101B5000DB5005E0130ED9EC11F001E26ADBFDEC7D
:101B600011F002E2130E37DBC0EC11F006E0040EB8
:101B7000D9EC11F002E2050E2EDB030EDBB005D02E
:101B8000FCDA01E0D7D2080EDB6A090EDB6A0E0E22
:101B9000DBCFF6FF0F0EDBCFF7FF100EDBCFF8FF2A
:101BA0000800F550DF6EDF5014E003EC12F011E294
:101BB00012EC12F003E1151C01E1BCD2BBDB01E326
:101BC000DB2A090EDB2AD9500E0FE96E000ECBDBA3
:101BD000E7D7D3DA01E1B4D2ADD2C6DA110EEECF37
:101BE000DBFF120EEDCFDBFF110EDBCFE6FF120E97
:101BF000DBCFE6FFB5EC17F0E552E552130EF3CF5D
:101C0000DBFF140EF4CFDBFF060EDB5004E0130EF7
:101C1000D0DB01E20EDBFDEC11F002E2130EDBDAA9
:101C2000AFDB05E0040EC5DB02E2050ED4DA030EDD
:101C3000DBB005D0A2DA01E07DD2080EDB6A090E26
:101C4000DB6A110EDBCFE9FF120EDBCFEAFFEFCF2D
:101C5000DFFFDF5014E0D7DB12E2E4DB03E1151C09
:101C600001E168D267DB01E3DB2A090EDB2A110EF2
:101C7000DB2ADBCFE9FF120EE8E3DB2AE6D77DDAC9
:101C800001E15ED257D2030EDB8E070EDB0410E1BA
:101C900095DB040E5ADB0A0EEECFDBFF0B0EEECF08
:101CA000DBFF0C0EEECFDBFF0D0EEECFDBFF6CD0BB
:101CB000070EDB5003082CE1030EDBAE0DD0B2DAC9
:101CC000020E76DAEFCF14F0156A166A176A14AEB0
:101CD00039D01568166835D0F70EDBCF15F0F80E41
:101CE000DBCF16F0020E155E000E165AF70E15C069
:101CF000DBFFF80E16C0DBFF15C0E9FF16C0EAFFD8
:101D0000EFCF14F00A0E14C0DBFF0B0EDB6A38D0E5
:101D1000070EDB50020809E1030EDBAE04D059DBED
:101D200016AE10D00ED055DB0DD0030EDBAE12D0A8
:101D300079DA020E3DDAF9DA166A176A15AE02D0C0
:101D400016681768E2DA0C0E16C0DBFF0D0E17C01E
:101D5000DBFF1AD0F70EDBCF16F0F80EDBCF17F053
:101D6000020E165E000E175AF70E16C0DBFFF80EB5
:101D700017C0DBFF16C0E9FF17C0EAFFD6DAC5DAE5
:101D80000C0EDB6A0D0EDB6A060EDB5005E1010E60
:101D9000F36E050EF3CFDBFF150EDB6A160EDB6A62
:101DA000D950370F146E000EDA20156E390E14C09C
:101DB000DBFF3A0E15C0DBFF380EDB6A080EDB6A6C
:101DC0000A0EAEDADF50780A12E0200A10E0280A84
:101DD0000CE0200A0AE03F0A06E00D0A02E0200AB1
:101DE00008E1020E05D0080E03D0080EDF26100E03
:101DF00097DA030EDBBE02D0DB92DB94DB50800B64
:101E000024E08ADAD890030EEB50000A08E6000EB0
:101E1000EE5C000EEE58000EEE58000EEE5815E285
:101E200013DA09680A680B680C6863EC18F00A0E8C
:101E300000C0DBFF0B0E01C0DBFF0C0E02C0DBFF9E
:101E40000D0E03C0DBFF2D0E08D0030EDBA202D067
:101E50002B0E03D0DBA408D0200EF36E170EF3CFA9
:101E6000DBFF150EDB2A02D0170EDB6A050EDB50F6
:101E700003E1B7D901E189D03E0E146E330E156E21
:101E8000000E166E070EDBCF17F0186A196A1A6A71
:101E900017C009F018C00AF019C00BF01AC00CF0F6
:101EA000D3D99BEC18F014500024F36E1550012088
:101EB000F46E16500220F86EF4CFF7FFF3CFF6FF62
:101EC0000800090EF5CFDBFF580EDF5C0FE1610E55
:101ED000F36E090E7BD90AE3200E146E090EDBCFD8
:101EE000E7FF1450E75E090EE7CFDBFF070EDBCFFD
:101EF00014F0156A166A176A0FDA14C009F015C0D3
:101F00000AF016C00BF017C00CF0EECF04F0EECFC5
:101F100005F0EECF06F0EFCF07F09BEC18F007C00E
:101F2000EDFF06C0EDFF05C0EDFF04C0EFFF390E69
:101F3000DBCFE9FFDB063A0EDBCFEAFF01E2DB068F
:101F4000090EDBCFEFFF150EDB2A4BD995E1030E0F
:101F5000DBA61DD06F0EDF5C06E1C1D918E3150EBC
:101F6000DB285BDA14D0780EDF5C09E0580EDF5C0A
:101F700006E0620EDF5C03E0420EDF5C08E1020E69
:101F8000F36E160EF3CFDBFF02D0150EDB6A030EE5
:101F9000DB50100B0EE0040EDBCF14F0050EDB500F
:101FA000D880145406E2060EDB5003E1040EDB5029
:101FB00034DA95D90AE2050EDBCFE7FF150EDB50C8
:101FC000E75E050EE7CFDBFF02D0050EDB6A040EED
:101FD000DBCF14F0160E45D9D880145414E2160E37
:101FE000DBCFE6FF150EDBCFE6FF040EDBCFE6FF0F
:101FF000050EDB50E552E75CE552D880E754E55228
:10200000D880E7545FD9030EDB50010B0BE1080EBB
:10201000DB5008E0B2D801E08DD0080EDB50BED80E
:10202000080EDB6A170EDB5007E088D9170EF1D9CE
:1020300003E1151C01E17ED0160EDB5016E07ED9BF
:10204000300EE66E9FD802E1151C74E077D9DFCF21
:10205000E6FFE8EC17F0E552E552E552F4CF15F053
:102060000001F31C02E1151C65E0050EDBCF14F046
:10207000160EDB50D880145409E2050EDBCFE7FFC3
:10208000160EDB50E75E050EE7CFDBFF300EE66E87
:10209000050ECBD94FE1390EDB2ADBCFE9FF3A0E33
:1020A00001E3DB2ADBCFEAFF090EEFCFDBFFDB50DA
:1020B0000EE044D9090EADD902E1151C3BE0390E02
:1020C000DB2ADBCFE9FF3A0EEDE3DB2AEBD755D86D
:1020D00031E1160EDBCFE6FF080EC3D8E552E72448
:1020E0005DD82ED0070EDB50030A1CE0010A14E075
:1020F000030A07E07BD9DBCFEEFF020EDBCFEDFF5B
:102100001FD0F5D8196A17AE02D0186819682CD8F4
:10211000BCD819C0EEFF14D0EAD817BE186824D86E
:10212000B4D80ED063D9DBCFEFFF0AD07BD905E15D
:10213000151C03E1F368F46810D0FCD801E3DB2A36
:1021400079D93FEF0CF0010EDBCF14F0020EDBCF9C
:1021500015F014C0F3FF15C0F4FF3B0EE15C02E282
:10216000E16AE552E16ECBD029D9020EA5EF11F05C
:1021700061D90800F550DF6E1200200EE66E080EE1
:1021800015EF12F0E8EC17F0E552E552E552F3CF07
:1021900014F0F4CF15F00001F31C1200146E156A50
:1021A000D950010F4DD91450EE261550ED221200D2
:1021B000185E000E195AF70E18C0DBFFF80E19C092
:1021C000DBFF18C0E9FF19C0EAFF1200DBCFF4FF04
:1021D000F350F45C1200DB50E76E040EE7CFDBFF38
:1021E00012000A0EDBCF14F00B0EDBCF15F00C0E35
:1021F000DBCF16F00D0EDBCF17F0145015101610B4
:1022000017101200130EEECFDBFF140EEDCFDBFF25
:10221000130EDBCF14F0140EDBCF15F00001800E8F
:1022200015141200F70EDBCF18F0F80EDBCF19F003
:102230001200050EDB50E66ED950130F01D9E5529E
:10224000E750EE6EED6A12000A0EDBCF04F00B0EC3
:10225000DBCF05F00C0EDBCF06F00D0EDBCF07F069
:102260001200DBCFE6FF150EDBCFE6FF050EDB50DD
:10227000E552E724E552E7241200DB50CED8010EE8
:10228000F36E060EF3CFDBFF1200EE50EFCFEAFF46
:10229000E96E16C0EEFF17C0EEFF18C0EEFF120089
:1022A000D9CFE6FFDACFE6FFE1CFD9FFE2CFDAFF01
:1022B0001200DFCFE6FFE66A61EC19F0E552E55265
:1022C000F3501200E76E080EE7CFDBFF1200EECFEF
:1022D00014F0EECF15F0EFCF16F0176A1200050ECE
:1022E000DBCF14F0150EDB50D88014541200010E11
:1022F000DBCF16F0020EDBCF17F0186A1200E552A2
:10230000E5CFDAFFE7CFD9FF12000A0E14C0DBFFDA
:102310000B0E15C0DBFF1200D9500A0F20EF12F090
:10232000F36E070EF3CFDBFF1200EECF14F0EFCF0A
:1023300015F01200010EDB2A020E1200FC0EDBCF9C
:10234000E6FFFD0EDBCFE6FF1200145E000E155A0D
:10235000F70E14C0DBFFF80E15C0DBFF14C0E9FF59
:1023600015C0EAFF1200DA20EA6EEF2AEECFF6FF80
:10237000000EEF22EECFF7FFEF22EECFF8FF1200B4
:10238000040EDBCFE6FF130EDB50E552E75C9ADF6D
:10239000DB5004DF060EDB501200090EDB500A0D85
:1023A000F350DF24D00FE76E090EE7CFDBFFB8EF65
:1023B00010F0DB50F36E050EE6EF10F0F70EDBCFFA
:1023C00014F0F80EDBCF15F01200DFCFE6FFC2EFFE
:1023D00010F028DF030EECDE67EF11F014EC0CF0C8
:1023E000E552E552E552E55200091200BDDEEE501D
:1023F000EFCFEAFFE96E010E1200130EDB50F36E11
:10240000040EE6EF10F0040EDB50F36E090EE6EF5B
:1024100010F0DBCFE6FFC2EF10F0E76E050EE7CF5E
:10242000DBFF12008BDFE5EF11F0DBCFE6FF86DF8D
:10243000EEEF11F0D950F90FE96EFF0EB3EF11F086
:10244000E96E000EDA20EA6E12000F9E08D00F9E91
:1024500007AE05D0066C071EE86A07220F8E07C07C
:1024600001F006C000F0136A126A8E0E026E036A53
:102470005EEF14F00F9E0CD00F9E07AE09D0046CD7
:10248000051E061E071EE86A0522062207220F8E79
:1024900007C001F006C000F005C013F004C012F040
:1024A0009E0E026E036A5EEF14F00D7E0F6A9AECC8
:1024B00014F0B2EC14F00FB642EF14F00FA20AD0F1
:1024C0000FAA03D00FBE42EF14F00FA44EEF14F08A
:1024D0004BEF14F00FAA05D00FAC4EEF14F04BEFFA
:1024E00014F00FA00AD00FA808D00FBE04D00FA47C
:1024F00002D057EF14F05BEF14F0126A036A0D502C
:10250000085C116E10E305C013F006C000F007C0B0
:1025100001F008C010F00AC005F00BC006F00CC0B6
:1025200007F00F3A09D00AC013F00BC000F00CC03E
:1025300001F00DC010F0116C0F9E0FBC0F8E10C07B
:1025400002F00FB08AEF14F01A0E11608AEF14F047
:10255000026A086A0FA408D0056C061E071E081E32
:10256000E86A0622072208220FAC08D0136C001E6E
:10257000011E021EE86A002201220222046A115290
:1025800007E008340732063205320432112EF9D73B
:10259000055013260650002207500122085002223F
:1025A00004C012F00F9E02AE0BD0126C131E001E60
:1025B000011E021EE86A13220022012202220F8E4F
:1025C00002A006D0D8800132003213321232102A13
:1025D00010C002F05EEF14F00F6A9AEC14F0B2EC47
:1025E00014F00FB642EF14F00FA205D00FBA42EF6D
:1025F00014F049EF14F00FBA55EF14F00FA005D006
:102600000FB842EF14F055EF14F00FB849EF14F083
:10261000036A7F0E0824026EE86A03220D50025EF0
:10262000E86A035A1A0E106E086A126A136A006A80
:10263000016A0A50055E0B50065A0C50075A000EEC
:10264000085A09E70A5005260B5006220C500722AB
:10265000000E082201D0128AD890053606360736B9
:102660000836D8901236133600360136102EE1D7D0
:10267000075006100510D8A4128A5EEF14F00F6AF6
:102680009AEC14F0B2EC14F00FB642EF14F00FA273
:1026900005D00FB842EF14F049EF14F00FAA05D09F
:1026A0000FB042EF14F049EF14F00FB002D00FA8B2
:1026B00002D055EF14F0036A0D500824026EE86A48
:1026C00003227E0E025EE86A035A126A136A006AE7
:1026D000016A0C500702F4CF01F0F3CF00F00B5069
:1026E0000702F3501326F4500022000E01220C5072
:1026F0000602F3501326F4500022000E01220A5065
:102700000702F3501226F4501322000E0022012279
:102710000B500602F3501226F4501322000E002232
:1027200001220C500502F3501226F4501322000E21
:10273000002201220A500602F4501226000E132233
:10274000002201220B500502F4501226000E132223
:10275000002201225EEF14F00F6A9AEC14F00FB61B
:10276000B6EF13F00FA20ED00FB405D07F0E076E98
:10277000FF0E066E1FD0800E076E066A1BD0076A1A
:10278000066A18D00FB0FBD78F0E0860EDD77E0E0B
:102790000864F5D78E0E085C05E0D8900732063243
:1027A000082AF8D70FA406D0066C071EE86A07228D
:1027B00007AEE5D71200EDEC13F00FB6000C0FB02A
:1027C000000C0FB4000C010CEDEC13F00FB6000C74
:1027D0000FB0000C0FA4000C010C0F6A9AEC14F05F
:1027E000B2EC14F00FB612000FAE08D00FA004D058
:1027F0000FA802D00F8012000F9012000D50085C3D
:102800000BE10C50075C08E10B50065C05E10A5037
:10281000055C02E10F801200D8A002D00F8E10D00C
:1028200008500DC008F00D6E07500CC007F00C6E7C
:1028300006500BC006F00B6E05500AC005F00A6E7C
:102840000D50085C10E0FF0F09E00F900FB403D0AB
:102850000FAE0F8412000FAE0F9412000D2AD89005
:102860000C320B320A320A50055E0B50065A0C50DD
:10287000075A07BEEAD7D890053606360736082E1F
:10288000F8D7C8D77F0E086EFF0E076E066E056E6E
:1028900012007F0E0FBEFF0E086E02D07F0E086E74
:1028A000800E076E066A056AF3D70FAE04D0800E5D
:1028B000086E076AF7D7086A076AF4D70150001054
:1028C00013101210F8E003BEF0D701BE0CD0025076
:1028D0000310EBE0D89012361336003601360206AC
:1028E000D8A00306F2D70350D4E10228D2E012AEFA
:1028F00011D07F0E121402E113A00CD0132AE86A43
:102900000022012207E3D880013200321332022A6A
:102910000228BFE00250C9E013C005F000C006F075
:102920000134076E0230086E0732089E0FBE088E13
:1029300048EF14F00736083602E30F840F7E06E1F5
:102940000F80086A076A066A056A1200082803E011
:10295000D88007321200D890073202E10F821200AD
:102960000F8612000C360D3602E30F8C0F7E06E147
:102970000F880D6A0C6A0B6A0A6A12000D2803E0C0
:10298000D8800C321200D8900C32EAE10F8A120083
:1029900007C013F006C012F006500B02F4CF05F08A
:1029A000F3CF04F007500C02F4CF07F0F3CF06F09A
:1029B0000B02F3500526F4500622E86A0722125053
:1029C0000C02F3500526F4500622E86A07220CAEEA
:1029D000EEEF14F01250065E1350075A13AE000CBF
:1029E0000B50065E0C50075A000C008080808080DF
:1029F000800000C0C0C0C0C0C00000E0E0E0E0E077
:102A0000E00000F0F0F0F0F0F00000F8F8F8F8F86E
:102A1000F80000FCFCFCFCFCFC0000FEFEFEFEFEE0
:102A2000FE0000FFFFFFFFFFFF000010181C1E1C30
:102A30001810000103070F070301040E1F0E0E0EEE
:102A40000E0E0E0E0E0E0E1F0E0402040E111F109F
:102A50000E0008040E111F100E0008040E010F11C5
:102A60000F00020502000000000050726F6A6574DA
:102A700020617665632050494331384632364B3207
:102A800032202B204C434431783136202B204D61AD
:102A90007833323332200D0A005061746820433A93
:102AA0005C5F4331385C5F4D657350726F6A65746B
:102AB000735F4331385C467265715F506572696F50
:102AC000640D0A0056657273696F6E3A2031352DB8
:102AD00031312D323031330D0A20506F7274206342
:102AE0006F6D6D203139323030626473206F7576CE
:102AF00065727420513D32304D687A0D0A002046CF
:102B000072657175656E63656D65747265203148B7
:102B10007A202E2E203130204D487A2C20436F729F
:102B20007265637469662031207365636F6E6465D6
:102B3000203D20340D0A20002054696D657231203B
:102B400053414E53207072657363616C6572203D12
:102B500020636F6D7074657572206427696D707580
:102B60006C73696F6E73200D0A002054696D657275
:102B700030203D2066656E65747265206465206353
:102B80006F6D7074616765202C6261736520312000
:102B90007365632061766563205241323D31200DBB
:102BA0000A002054696D657230203D2066656E65AF
:102BB00074726520646520636F6D70746167652051
:102BC0002C626173652034207365632061766563D0
:102BD000205241323D30200D0A0046726571656E0B
:102BE00063656D6574726520202000313846323689
:102BF0006B323220513D32304D687A0067616D6D25
:102C0000652031487A2E2E31304D687A00313030CF
:102C100025204D504C41422043313820200076651C
:102C20007273696F6E3A31352D31312D3133004D6C
:102C30006573757220656E2031206F7520347300C6
:102C400056696120657461742064652052413220A8
:102C5000004C6F6E677565722064274F6E64653D2A
:102C60002000202020202020202020202020202084
:102C70002020007061756C666A756A6F2E667265D9
:102C8000652E6600D9CFE6FFDACFE6FFF80EE3CF78
:102C9000D9FFF90EE3CFDAFFE652E652E652E652EA
:102CA000E652FB0EE124E76EFF0EE220E46EE652F0
:102CB000F30EE3CFE6FFF30EE3CFE6FFF30EE3CF31
:102CC000E6FFF30EE3CFE6FFC7EC16F0F50EE124C6
:102CD000E96EFF0EE220EA6EB4EC16F019E1B7ECF3
:102CE00016F018E1B4EC16F017E1B7EC16F016E1A7
:102CF000B4EC16F015E1B7EC16F014E1B4EC16F0F4
:102D000013E1B7EC16F012E1B4EC16F011E112D0B9
:102D1000BDEC16F0C2EC16F0BDEC16F0C2EC16F0ED
:102D2000BDEC16F0C2EC16F0BDEC16F0C2EC16F0DD
:102D3000BDEC16F0C2EC16F0DE6AF50EE126FF0ED1
:102D4000E222FF0EE3CFDAFFE552FF0EE3CFD9FF19
:102D5000E552FA0EE124E96EFF0EE220EA6EEECFB4
:102D6000F3FFEFCFF4FF1200EF380F0B1200EF501C
:102D70000F0B02E1EE52D8841200EF380F0B300F28
:102D8000DE6E1200EE500F0B300FDE6E1200FA0EE8
:102D9000E3CFE9FFFB0EE3CFEAFF200EE66EEE6A1B
:102DA000EE6AEE6AEE6AEF6AD890FB0EE336FC0E2E
:102DB000E336FD0EE336FE0EE336ED36ED36ED3648
:102DC000ED36EF36FF0EE3060FE0F6EC16F0EE52AE
:102DD000F6EC16F0EE52F6EC16F0EE52F6EC16F0BB
:102DE000EE52F6EC16F0E1D7E56E1200030EEF247A
:102DF000E8B6EF6E300EEF24E8BEEF6E000C0E0E5C
:102E0000F66E000EF76E000EF86E01010900F55027
:102E1000FA6F0900F550FB6F03E1FA6701D03DD06E
:102E20000900F550F56F0900F550F66F0900F550EF
:102E3000F76F09000900F550E96E0900F550EA6ED8
:102E4000090009000900F550F86F0900F550F96F05
:102E500009000900F6CFFCF1F7CFFDF1F8CFFEF144
:102E6000F5C1F6FFF6C1F7FFF7C1F8FF0101F8530E
:102E700002E1F95307E00900F550EE6EF807F8E2B9
:102E8000F907F9D7FCC1F6FFFDC1F7FFFEC1F8FF56
:102E90000101FA07000EFB5BBFD71200D9CFE6FF96
:102EA000DACFE6FFE1CFD9FFE2CFDAFFE652E65212
:102EB000E652E652D950F90F146EFF0EDA20156E65
:102EC00014C0DEFFDD6EDECFE6FFDDCFE6FFF90EDC
:102ED000DBCFE6FFFA0EDBCFE6FFFB0EDBCFE6FF34
:102EE000FC0EDBCFE6FFFD0EDBCFE6FF2AEC0CF09D
:102EF000146E070EE15C02E2E16AE552E16E1450E5
:102F0000020EF3CFDBFF030EF4CFDBFF020EDBCFAD
:102F100014F0030EDBCF15F014C0F3FF15C0F4FF5F
:102F2000040EE15C02E2E16AE552E16EE552E5CFB2
:102F3000DAFFE7CFD9FF1200FB0EE3CFF6FFFC0E5E
:102F4000E3CFF7FFFD0EE3CFF8FFFE0EE3CFE9FF7F
:102F5000FF0EE3CFEAFFE9CFF3FFEACFF4FF09006A
:102F6000F5CFEFFFEE66FBD71200FE0EE3CFE9FFD1
:102F7000FF0EE3CFEAFFF36AF46AEE5203E0F34A8E
:102F8000F42AFBD71200FF0EE3CFF8FFE552FF0E45
:102F9000E3CFF7FFE552FF0EE3CFF6FFE552E66A17
:102FA000E66AE66A0900F55209E0FD0EE32A05E14A
:102FB000FE0EE32A02E1FF0EE32AF4D7FD0EE3CF73
:102FC00005F0FE0EE3CF06F0FF0EE3CF07F0120090
:102FD000D9CFE6FFDACFE6FFE1CFD9FFE2CFDAFFC4
:102FE000FB0EDBCF14F0FC0EDBCF15F00001800EE2
:102FF00015141AE1FB0EDBCFE9FFFC0EDBCFEAFF75
:10300000EECFF3FFEDCFF4FFEE2A000EEF22F3CF69
:10301000E9FFF4CFEAFFFD0EDBCFEFFFEF50156ABB
:10302000F36E15C0F4FF10D0FB0EDB50FE0806E176
:10303000FD0EDBCFE6FF91EC19F005D0FD0EDBCFE6
:10304000E6FF03EC00F0E552E552E5CFDAFFE7CF0B
:10305000D9FF1200D9CFE6FFDACFE6FFE1CFD9FFE3
:10306000E2CFDAFFAC6AAB6AFD0EDBB0AC88DBA264
:1030700002D0AC8CAB8CDBB4AC8EDBA602D0AB88C0
:1030800001D0AB8ADBB8AC84DBBAAB86DBAC02D058
:103090009D8A01D09D9ADBAE02D09D8801D09D987B
:1030A000FB0EDB50AF6EFC0EDBCF15F015C014F03D
:1030B000156A1450B06EAC8AAB8EE552E5CFDAFFDC
:1030C000E7CFD9FF120004500902F3CF00F0F4CF8C
:1030D00001F00A02F3500126000EF420026E0450A3
:1030E0000B02F3500226000EF420036E04500C0273
:1030F000F350032605500902F3500126F450022232
:10310000000E032205500A02F3500226F450032257
:1031100005500B02F350032606500902F350022615
:10312000F450032206500A02F35003260750090206
:10313000F35003261200036A026A016A006A200E35
:10314000E76ED89004360536063607360036013667
:10315000023603360950005C0A5001580B500258E1
:103160000C50035809E30950005E0A50015A0B50F5
:10317000025A0C50035A042AE72EE4D71200D9CF82
:10318000E6FFDACFE6FFE1CFD9FFE2CFDAFFE65282
:10319000F20E0101FF17ABAC03D0FF91ABB0FF8182
:1031A000ABB4FF85ABB2FF87AE50DF6EDF50E552A8
:1031B000E552E5CFDAFFE7CFD9FF1200D9CFE6FF1E
:1031C000DACFE6FFE1CFD9FFE2CFDAFFE652E652EF
:1031D000CE50DF6E010ECFCFDBFFDECF14F0DDCFA0
:1031E00015F014C0F3FF15C0F4FFE552E552E552A7
:1031F000E5CFDAFFE7CFD9FF1200D9CFE6FFDACF6C
:10320000E6FFE1CFD9FFE2CFDAFFE652E652FC0E4D
:10321000DBCFDEFFDBCFDDFF010EDB50CF6EDF50FB
:10322000CE6EE552E552E552E5CFDAFFE7CFD9FFA2
:103230001200D9CFE6FFDACFE6FFE1CFD9FFE2CF28
:10324000DAFFE652E652FC0EDBCFDEFFDBCFDDFF1E
:10325000010EDB50D76EDF50D66EE552E552E552D7
:10326000E5CFDAFFE7CFD9FF1200D9CFE6FFDACFFB
:10327000E6FFE1CFD9FFE2CFDAFFACAC04D0AC90EF
:103280000101FFB3AC80FD0EDB50AD6EE552E5CF22
:10329000DAFFE7CFD9FF12002563204F2E432E3DE2
:1032A000202573204D00256320502E4F2E3D2025D4
:1032B00073204D00256320472E4F2E3D202573207F
:1032C0004D00F36AF46AFF0EE124E96EFF0EE2207E
:1032D000EA6EED6607D02F0EEF6404D03A0EEF6071
:1032E00001D0F32A1200380EF36E00EE00F00F0E3C
:1032F00001D81200EA6002D0EE6AFCD7F350E96010
:103300001200EE6AFCD71EEE00F02EEE00F0F86A16
:103310000F9CFFEC16F0A8EC19F05AEC06F0FBD766
:103320001200FF0EE350ACBA04D0AF6AAB8EAC8A89
:10333000949CACA2FED7AD6EF36EF46A12003031ED
:10334000323334353637383961626364656600FF7D
:1033500012006A2A992AC42AFE2A382B6A2BA22B29
:10336000DA2BEB2BFC2B0D2C1E2C2F2C402C512C54
:10337000622C732C00003132333435363738393013
:10338000313233343536370000FFFFFFFFFFFFFFD8
:10339000FFFFFFFFFFFFFFFFFFFFFFFFFFFFFFFF3D
:1033A000FFFFFFFFFFFFFFFFFFFFFFFFFFFFFFFF2D
:1033B000FFFFFFFFFFFFFFFFFFFFFFFFFFFFFFFF1D
:1033C000FFFFFFFFFFFFFFFFFFFFFFFFFFFFFFFF0D
:0200000400F00A
:020000040030CA
:0E0000000022193C009D84000FC00FE00F404D
:020000040020DA
:08000000FFFFFFFFFFFFFFFF00
:00000001FF
